:100000000200EB320000000000000032000000009F
:10001000000000320000000000000032000000007C
:100020000000003200000000000000000000C39546
:10003000F02212002E60044002E422740122120019
:100040002E6003500122E42212005460044002E4B6
:1000500022740122C3EDB50706ECB50602E4227452
:100060000122AE02E6F70809DEFA22209802E42215
:100070003098FDE599C29822740D120083740A121B
:100080000083223099FDC299F59922F874AD0400DD
:100090000000000000000070F500D8F022E6F760D4
:1000A000040809DAF8E4F722E760030980FA22E697
:1000B00060061200830880F722E82A14F8AE02E6F0
:1000C0001200C918DEF9E4F722FCC41200CFEC5488
:1000D0000FC3940A400424418002243AF70922E61F
:1000E0002401F6FA08E63400F64A22787FE4F6D8CE
:1000F000FD758151C28E759852758922758DF4D225
:100100008E75200075B0FF7590FF7580FF75A0FF9C
:10011000753900A2B49204500302011F433901A2B1
:10012000B59204500302012B433902E539B40002B1
:10013000800302013802035675380051B6E534B425
:100140005402800302015B0538E538B403028002E3
:100150005003020158753803020177E534B43A02BE
:10016000800302017475F003E538113E600302015B
:100170007402017A75380002013B753A007106E598
:1001800034B40002800302018C02019CE534B539CD
:1001900002800302019902019C0201387106853434
:1001A0003B710685343C710685343D853A377106CE
:1001B000E537B5340280030201C00201C30201C366
:1001C0000201CC853B90853C80853DA030B7FDC2C7
:1001D000B27405118B74FFC0E0793ED0E0F7097767
:1001E0000074AAC0E0793E11A8D0E0F70977007941
:1001F0003E11A87B05EB04FB83F70970F8800752DA
:10020000525252523A0078397A01792111B9793E25
:1002100011A878217A1212009D85901478147A0121
:10022000792111B9793E11A878217A1212009D85A1
:10023000801478147A01792111B9793E11A87821B6
:100240007A1212009D85A01478147A01792111B9CF
:10025000793E11A878217A1212009D753A007538FE
:100260000975F010E538113270030202987A0174B2
:100270003EC0E08538F0D0E025F014F87934120063
:10028000628534F0E53A25F0C0E0783AD0E0F60532
:1002900038E5386003020261783A7A01792111B9B0
:1002A000793E11A878217A1212009D783E11AF1183
:1002B00078D2B20201387532007533007834116B90
:1002C000F6C2B37401118BE539B400028003020257
:1002D000E7783211DFAC32AD337ED07F0711486052
:1002E000030202E7020356D2B3E534B4000302036B
:1002F000028534F0E53A25F0C0E0783AD0E0F60225
:1003000003050202BC2251B671378534367836E6D1
:1003100023F67836E623F67836E623F67836E623B3
:10032000F65336F051B671378536F0E53445F0C0F6
:10033000E07834D0E0F62275F041E534113E6003F8
:1003400002035275F007E534C395F0C0E07834D06D
:10035000E0F653340F22C2B2740A118B74FFC0E06E
:10036000793ED0E0F709770074AAC0E0793E11A881
:10037000D0E0F7097700793E11A87B05EB04FB83F9
:10038000F70970F8800754545454543A0075140017
:1003900078147A01792111B9793E11A878217A125D
:1003A00012009D8590377837E623F67837E623F6F6
:1003B0007837E623F67837E623F643370F78377A2F
:1003C00001792111B9793E11A878217A1212009D84
:1003D00085A01478147A01792111B9793E11A87891
:1003E000217A1212009D7514FF78147A0179211177
:1003F000B9793E11A878217A1212009D753A0075DC
:10040000380975F010E538113270030204397A01A9
:10041000743EC0E08538F0D0E025F014F87934124D
:1004200000628534F0E53A25F0C0E0783AD0E0F695
:100430000538E5386003020402783A7A017921111F
:10044000B9793E11A878217A1212009D783E11AF39
:100450001178D2B275380051B6E534B45202800337
:100460000204770538E538B4030280025003020421
:1004700074753803020493E534B43A02800302042D
:100480009075F003E538113E600302049002049673
:10049000753800020457753A007106710685343BC1
:1004A000710685343C710685343D853A377106E521
:1004B00037B5340280030204BF0204C20204C20240
:1004C00004E2783BE623F6783BE623F6783BE62326
:1004D000F6783BE623F6433B0F853B90853D8075E0
:1004E000A0FF020356000000000000000000000012
:00000001FF
